:10000000180800107501000000000000000000004A
:10001000E1020000E1020000E10200000000000037
:10002000000000000000000000000000E1020000ED
:10003000E102000000000000E1020000E102000017
:10004000E1020000E1020000E1020000E102000024
:10005000E1020000E1020000E1020000E102000014
:10006000E1020000E1020000E1020000E102000004
:10007000E1020000E1020000E1020000E1020000F4
:10008000E1020000E1020000E1020000E1020000E4
:10009000E1020000E1020000E1020000E1020000D4
:1000A000E1020000E1020000E1020000E1020000C4
:1000B000E1020000E1020000E1020000E1020000B4
:1000C000E10200002DE9F04182B000F0D3F9254BA8
:1000D0004FF41641186800F067FA0127224D234CAF
:1000E0000026B8460222C5F81C800423AA61082213
:1000F000EB61AA6110232022EB61AA6140238022D8
:100100003146EB611A48AA6100F008FC0021019118
:100110000198711CA04205DC019A531C01930198BF
:10012000A042F9DD0223AF610422EB610823AA613A
:10013000EB6110222023AA61EB6140228023AA6197
:100140000B48EB6100F0EAFB0020019001990236B8
:10015000A142C7DC019A501C01900199A142F9DD2E
:10016000C0E700BF1400001040C00920FFFF0F00CF
:10017000EC0E0000684620F007018D46F1B500F056
:10018000B1F84F484F49884235D04F4CA14232D246
:10019000024652F8046B0B46CD4343F8046B6519D5
:1001A000A342C5F3810526D29DB1012D0BD0022DAE
:1001B00005D0156800F108021D6001F1080352F82E
:1001C000040B43F8040B52F8041B43F8041BA3422E
:1001D00011D296465EF8047B5668D568DEF80400B6
:1001E0009C464CF8047B5E60CCF80400DD60103364
:1001F0001032A342EDD335483549884234D0354CCE
:10020000A14231D2024652F8046B0B46CD4343F86B
:10021000046B6519A342C5F3810525D29DB1012D5B
:100220000BD0022D05D0156800F108021D6001F108
:10023000080352F8040B43F8040B52F8041B43F86C
:10024000041BA34210D294465CF8047B5668D56820
:10025000DCF80400194641F8047B5E604860DD600C
:1002600010331032A342EED31B491C48814221D2E5
:1002700000220B46CC4343F8042B04198342C4F3F9
:10028000810417D264B1012C06D0022C1CBF1A6065
:1002900001F1080343F8042B43F8042B834209D2ED
:1002A0009E464EF8042B5A60CEF80420DA601033D4
:1002B0008342F5D3FFF706FFBDE8F140854670475E
:1002C000240F0000000000100C000010240F00009C
:1002D00000000010000000100C00001018000010BA
:1002E000FEE700BF3649202330B4C1F8A031D1F871
:1002F000A001334A10F0400FF9D0324D0124AA205A
:1003000055230321C2F80411C2F80C411146C2F86A
:100310008450C2F88C00C2F88C30C2F88040C2F819
:100320008C00C2F88C30D1F88830254A13F0806FE9
:10033000F9D00321AA245520C2F88010C2F88C40BD
:100340001146C2F88C00D1F888301D4A13F0407F66
:10035000F9D02324C2F8A440AA2055230124C2F8CE
:10036000AC001146C2F8AC30C2F8A040C2F8AC00F4
:10037000C2F8AC30D1F8A830114A13F4806FF9D02C
:100380000321AA235520C2F8A010C2F8AC301146B0
:10039000C2F8AC00D1F8A800094A10F4407FF9D0A7
:1003A0000949002043F23A03C2F8A801C2F8AC019F
:1003B000C2F8C410C2F8C801136030BC704700BF57
:1003C00000C00F4063000500DE87280430B5254DCE
:1003D000254BD5F8C41083B041F08074C5F8C440F3
:1003E000D5F8C420002042F01001C5F8C4101A68E6
:1003F000044642F010051D60196821F020021A60C1
:100400001D6845F0400119601A6822F080051D60E2
:10041000196841F480121A601D6825F400111960F2
:100420001A6842F480051D601968104D21F400021D
:100430001A6000F097F90822012328604FF4164152
:10044000009400F071F9022000F08CF9084D4FF48F
:100450001641286008220123009400F065F903B0DA
:1004600030BD00BF00C00F4000C0024014000010AB
:100470000C000010104A10B5D2F8C4400F4B44F4E1
:100480000041C2F8C4101C686FF0FF0244F0FF0185
:1004900019600B48DA6100F06FF900F0FDF9094CC2
:1004A0002060094800F068F900F0F6F92060FFF7D5
:1004B0008DFF002010BD00BF00C00F4040C00920CC
:1004C000002D31011000001000879303024B0146FC
:1004D000186800F003B800BF14000010436913F05F
:1004E000200FFBD00160704730B42A4A84B00DF170
:1004F000040C04460D46284B07CAACE803009C4296
:100500008CF8002029D018DD244B9C421BD003F529
:1005100080418C4214D104A94D19214B15F80C0CC3
:10052000D3F8AC11820442EA0101C3F8AC11D3F84C
:10053000AC010240C3F8AC2102E01A4884421ED04C
:1005400004B030BC70470DF1100C6544144B15F825
:100550000C2CD3F8AC111204E5E704A94D19104B8B
:1005600015F80C0CD3F8A811020242EA0101C3F8F5
:10057000A811D3F8A8010240C3F8A821E0E70DF1C3
:10058000100C6544064B15F80C2CD3F8A8119201F9
:10059000EBE700BF080F00000000014000800940A9
:1005A00000C00F4000C000402DE9F047044682B073
:1005B0000F46002853D000F06FF9554E554B80463A
:1005C00030689C42019000F09C804BDD524B9C4275
:1005D0005DD003F5804294425FD0002302A800EB77
:1005E000030E1EF804CC3F01B8FBFCF3BB422BD238
:1005F000D6F80090474DDFF820A1AC42CDF804902A
:1006000067D050DC454B9C4235D000230DF1080EDD
:100610000EEB030C1CF8041C012920D049082046CD
:10062000FFF762FF3268AC4201925ED046DC3B4885
:10063000844226D0002302A901EB030E1EF804CC4D
:10064000B8FBFCF3BB42D8D3E268B3FBF7F342F04C
:100650008001E1602360E06820F08002E26002B087
:10066000BDE8F0872D498C42B7D12D48D0F8A8318C
:10067000C3F38113B2E72A48D0F8A821C2F381134B
:10068000C4E7274AD2F8A811C1F38113D3E724485D
:10069000D0F8AC31C3F30143A0E7214AD2F8AC1142
:1006A000C1F381439AE7544519D01E498C42ACD11D
:1006B0001B49D1F8AC31C3F38143A7E754451AD0A5
:1006C000184B9C42B6D1164BD3F8AC01C0F3814312
:1006D000B1E71349D1F8A831C3F3012396E71048D5
:1006E000D0F8AC21C2F3014390E70D4BD3F8A80139
:1006F000C0F301239FE70A4AD2F8AC11C1F30143CA
:1007000099E7074AD2F8A811C1F3012366E700BFB1
:10071000140F0000000001400080094000C00040AC
:1007200000C00F4000C0094030B4092A9DF80840BD
:100730000ED8013BDDB2053A012D0ED90023072C5E
:100740000ED900259C186419C46030BCFFF72CBF7B
:10075000013BDDB20322012DF0D89B00072CF0D81D
:10076000E500EFE703289ABF024B53F82000002072
:10077000704700BFF80E0000F0B4404D3F4CD5F874
:100780000C31D4F80C1113F0030F08BF3C4B3B4E57
:1007900001F003070CBF1A6842F21072D6F80C5130
:1007A000012F08BF374F05F0030308BF3A68022B3B
:1007B00008BF354B314908BF1A68344BB3FBF0F41E
:1007C000601EC1F804015000012218E0B4FBF0F1F2
:1007D000CF1F0132B7F5FC7F144622D9B5FBF0F1EB
:1007E000CD1F0132B5F5FC7F1BD9B6FBF0F1CD1F53
:1007F000A21CB5F5FC7F14D9E21C212A3BD0234969
:10080000234F244E5C18B3FBF0F1DD199E19CF1F66
:1008100003F18E4303F5060CB7F5FC7F0CF50C4392
:10082000D4D8541E154B220401398918AA24552006
:100830000122C3F88410C3F88C401946C3F88C0019
:10084000C3F88020C3F88C40C3F88C00D1F888002E
:100850000A4A10F0806FF9D00321AA205523C2F86C
:100860008010C2F88C001146C2F88C30D1F8882074
:1008700012F0407FFAD0F0BC704700BF00C00F40BC
:1008800004000010000000100800001000A3E11197
:100890000046C32300E9A4351C4A30B4D2F8845082
:1008A000D2F88440D2F80411D2F80C3113F0030FBF
:1008B00004BF174B1868154BD3F80C2102F0030C3A
:1008C000124ABCF1010FD2F80C2108BF114B02F003
:1008D000030C08BF1868BCF1020F04BF0E4B186868
:1008E0000A4BD3F8802012F0020F0CD0AA04930C0C
:1008F0005A1C5300C4F307444A1C00FB03F004FBDA
:100900000221B0FBF1F030BC704700BF00C00F40C7
:100910000400001000000010080000100FB42DE9C2
:10092000F04784B00CAB53F8045BDFF8FC803D4F1C
:1009300000240393287840B125280CD00135FFF717
:10094000C5FD287801340028F6D1204604B0BDE862
:10095000F04704B070476878013525285DD0253808
:10096000532855D8DFE810F09C025400540054007E
:1009700054005400540054005400540054005400D7
:1009800054005400540054005400540054005400C7
:1009900054005400540054005400540054005400B7
:1009A00054005400540054005400540054005400A7
:1009B0005400540054005400540054005400540097
:1009C00054005400540054005400540054005C017E
:1009D0005400540054005400540054005400540077
:1009E0005400540054016200540054005400540058
:1009F0005400540054005400540054005400540057
:100A00005400540054005400540054005400FB019E
:100A100003980135021D03928CE7FFF757FD01355E
:100A2000013487E767666666180F0000039BEC4693
:100A3000D3F8009098E80700ACE8030000200433E6
:100A400081456E4603938CF800208DF80900C0F2B2
:100A50002C82B9F1000F40F3D98087FB09204FEABF
:100A6000E971C1EBA00303EB830EA9EB4E0A0AF177
:100A700030098DF80090002B00F0208287FB03C91D
:100A8000DA17C2EBA90202EB820CA3EB4C03303362
:100A90008DF80130002A00F00E8287FB023ED0174D
:100AA000C0EBAE0303EB830AA2EB4A0130318DF8B1
:100AB0000210002B00F0048287FB03C9DA17C2EB97
:100AC000A90202EB820CA3EB4C0330338DF8033008
:100AD000002A00F0FB8187FB023ED017C0EBAE037B
:100AE00003EB830AA2EB4A0130318DF80410002B8E
:100AF00000F0E98187FB03C9DA17C2EBA90202EB18
:100B0000820CA3EB4C0330338DF80530002A00F043
:100B1000E08187FB023ED017C0EBAE0303EB830AF4
:100B2000A2EB4A0130318DF80610002B00F0D7817E
:100B300087FB03C9DA17C2EBA90202EB820CA3EB15
:100B40004C0330338DF80730002A00F0C58187FB55
:100B5000023ED017C0EBAE0303EB830AA2EB4A01BF
:100B600030318DF80810002B00F0BC8187FB03C9E1
:100B7000D817C0EBA90202EB820CA3EB4C03303375
:100B80008DF809304FF0090A16F80A00FFF79EFCAD
:100B9000BAF1000F0AF003030AF1FF3936DDD3B1D1
:100BA000012B0DD0022B05D016F80900FFF78EFCA3
:100BB00009F1FF3916F80900FFF788FC09F1FF3940
:100BC00016F8090009F1FF39FFF780FC09F1010C63
:100BD000BCF1000F1ADD16F8090009F1FF3AFFF722
:100BE00075FC16F80A00A9F1020AFFF76FFC16F867
:100BF0000A00FFF76BFCA9F10303F05CA9F10409FB
:100C0000FFF764FC09F101010029E4DC013591E6FC
:100C1000039A0135111D10780391FFF757FC89E6FF
:100C200003996E460A68081D02F00F03092B88BF5E
:100C30000733039098E8030086E80300111101F0E0
:100C40000F003033092888BF07300A118DF80030B3
:100C500002F00F033030092B88BF073311118DF8D4
:100C6000010001F00F00092888BF0730091101F0C9
:100C70000F023030092A88BF073203F130090B1107
:100C80008DF8030003F00F00092888BF07301B11FF
:100C900002F1300C03F00F02092A00F1300188BF85
:100CA0000732C3F303103032092888BF07303030D1
:100CB0008DF802908DF804C08DF805108DF806208F
:100CC0008DF80700082300E04B4603F1FF3916F8C2
:100CD00009003028F8D0002B98DDFFF7F7FBB9F1B9
:100CE000000F09F0030309F1FF3A8FDDD3B1012BA7
:100CF0000DD0022B05D016F80A00FFF7E7FB0AF12A
:100D0000FF3A16F80A00FFF7E1FB0AF1FF3A16F87E
:100D10000A000AF1FF3AFFF7D9FB0AF101010029A5
:100D20007FF774AF16F80A000AF1FF39FFF7CEFB20
:100D300016F80900AAF10209FFF7C8FB16F8090026
:100D4000FFF7C4FBAAF10303F05CAAF1040AFFF762
:100D5000BDFB0AF1010CBCF1000FE3DC56E703997F
:100D60006E460A68081D02F00F03092B88BF27335F
:100D7000039098E8030086E80300111101F00F00CA
:100D80003033092888BF27300A118DF8003002F06F
:100D90000F033030092B88BF273311118DF8010064
:100DA00001F00F00092888BF2730091101F00F0258
:100DB0003030092A88BF273203F1300C0B118DF82F
:100DC000030003F00F00092888BF27301B1102F130
:100DD000300903F00F02092A88BF27328DF802C0BC
:100DE00000F1300CC3F303103032092888BF2730DC
:100DF00030308DF804908DF805C08DF806208DF800
:100E00000700082300E04B4603F1FF3916F80900FC
:100E10003028F8D0002B7FF7F9AEFFF757FBB9F178
:100E2000000F09F0030309F1FF3A7FF7EFAED3B1EA
:100E3000012B0DD0022B05D016F80A00FFF746FB58
:100E40000AF1FF3A16F80A00FFF740FB0AF1FF3AF1
:100E500016F80A000AF1FF3AFFF738FB0AF101031E
:100E6000002B7FF7D3AE16F80A000AF1FF39FFF71F
:100E70002DFB16F80900AAF10209FFF727FB16F867
:100E80000900FFF723FBAAF10303F05CAAF1040AAF
:100E9000FFF71CFB0AF1010CBCF1000FE3DCB5E627
:100EA00025200135FFF712FB44E52D20C9F100098B
:100EB000FFF70CFBCDE54FF0010A65E69A4663E6C5
:100EC0004FF0020A60E64FF0040A5DE64FF0030AB5
:100ED0005AE64FF0050A57E64FF0070A54E64FF07E
:100EE000060A51E64FF0080A4EE600BF74657374B7
:100EF000202564200A0D000000C0004000000140D1
:100F00000080094000C00940010102020000000009
:100F100003000000040102082020202020202020BF
:040F200000000000CD
:0C0F2400001BB70000093D000080000029
:00000001FF
